:0300000002497141
:0C49710078FFE4F6D8FD7581740249B8A7
:101F67000A53746172743A20004950436F6E6E656C
:101F770063745245510A004950436F6E6E6563742E
:101F8700003E432C562C43432CC0E4E0EFF2E5F02F
:101F970020D1E8EDEAEEEC49500A003E432C4D41D2
:101FA700432C25303262583A25303262583A253070
:101FB7003262583A25303262583A25303262583AFE
:101FC70025303262582C4D414320E0E4F0E5F10A18
:101FD700003E432C5645522C20332E3020EEF22063
:101FE70025732025732CC2E5F0F1E8FF2049502026
:101FF700ECEEE4F3EBFF0A004F637420303320323A
:102007003030370031323A30313A3432003E432CE7
:102017004C442C50524F473A20202020202020208B
:1020270020202020202020202020202020202020A9
:102037002020202020202020202020202020202099
:102047002020202020202020202020202020202089
:10205700202020202020202020202020202CC4E009
:10206700F2E020EFF0EEF8E8E2EAE828F4E0E9EB46
:10207700290A003E2A2C312CCEF1EDEEE2EDFBE5EC
:1020870020EFE0F0E0ECE5F2F0FB20F1E5F2E5E22D
:10209700EEE3EE20E8EDF2E5F0F4E5E9F1E00A0021
:1020A7003E412C4130312C2562752E2562752E2537
:1020B70062752E2562752C495020E0E4F0E5F12089
:1020C700E0E4E0EFF2E5F0E00A003E412C41303277
:1020D7002C2562752E2562752E2562752E25627553
:1020E7002C495020E0E4F0E5F120EEF1ED2E20F14F
:1020F700E5F0E2E5F0E00A003E412C4130332C25C3
:1021070062752E2562752E2562752E2562752C49FE
:102117005020E0E4F0E5F120F0E5E72E20F1E5F0CE
:10212700E2E5F0E00A003E412C4130342C2562758F
:102137002E2562752E2562752E2562752CCCE0F151
:10214700EAE020F1E5F2E80A003E412C4130352C67
:102157002562752E2562752E2562752E2562752CD2
:10216700D8EBFEE70A003E532C4130362C2562752A
:102177002CC2F0E5ECFF20EEE6E8E42E20EAE2E8E8
:10218700F2E0EDF6E8E820282A3130ECF1290A00E0
:102197003E2A2C312CC4EEEF2E20EFE0F0E0ECE5E8
:1021A700F2F0FB20F1E5F2E5E2EEE3EE20E8EDF2F6
:1021B700E5F0F4E5E9F1E00A003E422C5330312C1A
:1021C7002562752CC6E4E0F2FC20E7E0EFF0EEF1C3
:1021D700E020F1EEE5E4E8EDE5EDE8FF20EEF220A2
:1021E700F1E5F0E2E5F0E00A003E422C5330322CF4
:1021F7002562752C43E2FFE7FC20F120F1E5F0E2D0
:10220700E5F0EEEC20EDE520EFEEE4E4E5F0E6E8BE
:10221700E2E0F2FC0A003E422C5330332C25627573
:102227002CCFE5F0E5E7E0EFF3F1EA20EFF0E82067
:10223700EFEEF2E5F0E520F1E2FFE7E820F120F12B
:10224700E5F0E2E5F0EEEC0A003E422C5330342C88
:102257002562752CCDE5F220EFE5F0E5E4E0F7E83F
:1022670020E4E8E0E3EDEEF1F2E8EAE820E220F12D
:10227700E5F0E2E5F00A003E422C5330352C2562AA
:10228700752CCAE0EDE0EB20F8E8F0EEEAEEE2E5C7
:10229700F8E0F2E5EBFCEDEEE3EE20EEE1ECE5ED48
:1022A700E00A003E532C5330362C25303262582535
:1022B7003032625825303262582530326258253024
:1022C70032625825303262582C4D414320E0E4F009
:1022D700E5F120F8E8F0EEEAEEE2E5F8E0F2E5EB0A
:1022E700FCEDEEE3EE20EEE1ECE5EDE00A003E4525
:1022F7004E440A0044756D7058202020202030304D
:102307002030312030322030332030342030352017
:1023170030362030372030382030392030412030D7
:10232700422030432030442030452030460A003ACE
:1023370020000A0044756D70442020202020303092
:1023470020303120303220303320303420303520D7
:102357003036203037203038203039203041203097
:10236700422030432030442030452030460A004583
:102377007272206B657900526420656570726F6DAB
:102387000A005264204D454D0A00526420436F6491
:10239700650A0044656275674950204F4E0A00443C
:1023A700656275674950204F46460A004465627565
:1023B7006755736572204F6E0A00446562756755ED
:1023C700736572204F46460A0044656275674D7310
:1023D70067204F6E0A0044656275674D7367204F2B
:1023E70046460A00436F6E666967206C6F636B2110
:1023F7000A00577220656570726F6D0A002053617D
:10240700766520656570726F6D210A0045727220CE
:102417004D414321004C6F61643E3E002A003C4120
:1024270030313D003C4130323D003C4130333D00CE
:102437003C4130343D003C4130353D003C41303675
:102447003D004E4F4950004C494E4B434F4E54525E
:10245700005452415353004652004E4F4C494E4B85
:1024670000494E49004E4F4449414700003C210076
:102477003C5330313D003C5330323D003C53303308
:102487003D003C5330343D003C5330353D003C5318
:1024970030363D00FF2449FF244EFF2458FF245EB9
:0C24A700FF2461FF2468FF246CFF2473F5
:0653BE00010B00010900D3
:10537A00C2AFC28E758900438910758BFF758DB7D0
:07538A00D2ABD28ED2AF229C
:03001B0002484B4D
:10484B00C0E0C083C082C0D0C2AFC28E758BFF7573
:10485B008DB720160675A61E75A6E10509D212E5C1
:10486B000B6002050BE50AD394014002150A050EF5
:10487B00E50E540F704AD21DE50E543F7014D21042
:10488B00907B09E0600C04F0E0D394B44004C2AF19
:10489B0080FE907B04E0600204F0907580E0600283
:1048AB0014F0907B0AE0D394014003E014F0301530
:1048BB0002050CE50DD394644004D2168002050D5D
:1048CB00E508D3940140021508D28ED2AFD0D0D0D8
:0648DB0082D083D0E03220
:10194F00C291C290D2B5C21A7D027C007F0712539A
:10195F000E8F26E526646060097D017F601252A21A
:10196F00D21AE4FDFC7F0B12530E8F26E52630E6CC
:10197F00097D04E4FF1252C6D21A7D017C007F0755
:10198F0012530E8F26E5267008FD7FFF1252A2D24A
:10199F001A301A03126000C2AFC288C2A8C2AA12BC
:1019AF004C069077BDE0B4FA09A3E064CE70030251
:1019BF001A46E4F52674B52526F582E43477F583C7
:1019CF00E4F00526E526B443EC9077BD74FAF0A356
:1019DF0074CEF0A374CCF09077C3740AF0E4A3F044
:1019EF00A304F0A3F09077C87403F0A374CCF09025
:1019FF0077B974FFF0A3F0A3F0E4A3F09077D47459
:101A0F0005F0E4F526E5262401FFE433FE74B52541
:101A1F0026F582E43477F583E0FD1253610526E560
:101A2F0026C3944340DFE4F5A775A61E75A6E19083
:101A3F007FF0F0A3F080FED2AF9077C87403F0A3CD
:101A4F0074CCF0E49077C7F012442CEF600312359A
:101A5F00BDC2B51233B6C2161250439077D4E0C34D
:101A6F00940350037403F0D21CD21BD21AD29320CA
:101A7F001A077E1F7F67124512E49079F4F0125314
:101A8F007AC2AFA37408F09077337424F0E4A3F014
:101A9F009077BDE0907735F09077BEE0907736F095
:101AAF009077BFE0907737F09077C0E0907738F07D
:101ABF009077C1E0907739F09077C2E090773AF065
:101ACF00750A01E49079F6F0C217C218D2AF75A764
:101ADF000775A61E75A6E112527C201A19AF267E35
:101AEF00007D031245F3E4FF1247A17E777FF4E4F4
:101AFF00FB7D011246CD907B09E060037401F0E499
:101B0F00907580F0A37455F0A37481F0E4F50CE4A4
:101B1F00F50D907580E07003122B87907B0AE0B46F
:101B2F0001119080007410F0E4907B0AF0D21AD269
:101B3F001BD21C908008E0F52630E405D2177410F4
:101B4F00F0E52630E508D2199080087420F0E526DC
:101B5F0030E608D2189080087440F0E50CD3940357
:101B6F004023908002E4F0908001F0908000F0E537
:101B7F000CD39406400FE4F50CC2139079F6F07570
:101B8F000A011250439080A0E07003124CFF908026
:101B9F00B8E07003124D799080D0E07003124EC1FF
:101BAF00908000E070133017101243289077B0EF39
:101BBF00F0D39400400312110C908002E070069055
:101BCF008000E06005D215021B1EC215E4F50C90D3
:101BDF007580E06003021B1E301912123E2A9077A7
:101BEF00B0EFF0D394004005E0FF1253912018039B
:101BFF00021D7D123CB59077B0EFF07003021B1EF3
:101C0F009077F4E054BF247F7003021CE01470033C
:101C1F00021CB824026003021D13201A077E1F7FC7
:101C2F0070124512301E792013769077CCE0700633
:101C3F009077D0E0605B907B00E0FF9077CCE0B5D1
:101C4F000724907B01E0FE9077CDE0B50618907BDE
:101C5F0002E0FE9077CEE0B5060C907B03E0FE909D
:101C6F0077CFE06E602B9077D0E06F7033907B0171
:101C7F00E0FF9077D1E0B50727907B02E0FF9077E8
:101C8F00D2E0B5071B907B03E0FF9077D3E0B50759
:101C9F000F9079F67401F0120021750A01021D7D73
:101CAF00907B0074FFF0021D7D907B09E060037450
:101CBF0001F0907AF8E0FF9077F6E06F6003021D75
:101CCF007D907AF8E004F0E4F50A9079F4F0021DC3
:101CDF007D301303021D7D9077C3E07003021B1E3E
:101CEF001253C5D213E4F50A9079F4F0907B0404F3
:101CFF00F0E4907AF7F0A3F0201A737E1F7F7E1224
:101D0F004512806A907B09E060037401F030135232
:101D1F009077F4E020E74B9077F6E0FF907AF7E0CA
:101D2F00FE6F600D907AFFE07007EE146F703F80CA
:101D3F0013907AF7E004F09077B0E0FFD39404406B
:101D4F000312513B90747C7482F0A37401F090776E
:101D5F00F6E090747EF07E747F7C7D03124C8402DB
:101D6F001B1E301E09201306907B0074FFF02013FA
:101D7F0003021E32E50A706B125179EF60207E78F4
:101D8F007FF49078F5E02404FD124C84907AFFE004
:101D9F006003021B1E9077D4E0F50A021B1E907B96
:101DAF0004E0D3943C403C907AFFE07036907B0483
:101DBF0004F0907732E0702B1253ABE49078F4F08C
:101DCF00A37412F0907AF8E09078F6F0A374FDF017
:101DDF0090758363A2019078F863A2017F12123885
:101DEF008B809B1253A0EF601590747C7483F0E48A
:101DFF00A3F07E747F7C7D02124C84021B1EE50AC9
:101E0F0064016003021B1E9079F4E004F0E0C394B8
:101E1F00055003021D8DC213E49079F6F0120021D4
:101E2F00021B1EE50A64016003021B1E9079F6E097
:101E3F0014604024FE603C147003021F1A240460D7
:101E4F0003021B1EE4F50C201E139079F67404F0A8
:101E5F009079F4E05401F0750A01021B1EE49079A9
:101E6F00F6F09079F404F0750AC8907B0074FFF0D7
:101E7F00021B1E907B00E07003021F099078F47420
:101E8F0080F09078F67401F0E4A3F0A304F0A3744B
:101E9F0030F0A3747BF0E4F52674FB2526F582E47D
:101EAF003478F583747DF074FC2526F582E434785C
:101EBF00F583E4F0E52624079078F5F07C7B7D0030
:101ECF009077C8E0FAA3E0FB7F02124A827E787F08
:101EDF00F4E5262409FD124C84907AFFE0601B1272
:101EEF0053C5D213E4F50A9079F4F0907B0404F013
:101EFF00E4907AF7F0A3F0021B1E9079F67404F0C9
:101F0F009077D4E02432F50A021B1E9080027410E1
:101F1F00F0750A039079F4E06401FFF09079F6749C
:101F2F0001F0EF70199077D0E06013FCA3E0FDA3F0
:101F3F00E0FEA3E0FF907B001225FC021B1E9077B2
:101F4F00CCE0FCA3E0FDA3E0FEA3E0FF907B00123A
:071F5F0025FC021B1E80FEA1
:011F66002258
:10110C009077F5E0B444047F0180027F009077F47F
:10111C00E0B447047E0180027E00EE5F604A907767
:10112C00BDE09077F6F09077BEE09077F7F090778F
:10113C00BFE09077F8F09077C0E09077F9F0907777
:10114C00C1E09077FAF09077C2E09077FBF090775F
:10115C00F57452F090772C63A2019080A863A201E1
:10116C007F0612388B0219459077B0E0C394085073
:10117C000302194E9077BDE0FF9077F6E06F6003A5
:10118C0002194E9077BEE0FF9077F7E06F60030294
:10119C00194E9077BFE0FF9077F8E06F600302196B
:1011AC004E9077C0E0FF9077F9E06F600302194E24
:1011BC009077C1E0FF9077FAE06F600302194E90D0
:1011CC0077C2E0FF9077FBE06F600302194E9077D7
:1011DC00F5E0B4441590772CE0B4FF0E63A20190B7
:1011EC0080A863A2017F0612388B907B09E0600314
:1011FC007401F0907B0A7464F09077F57452F0905F
:10120C0077F4E0646D60030213897BFF7A1F7988A1
:10121C0012288D7BFF7A1F79A29077BDE0F52FA362
:10122C00E0F530A3E0F531A3E0F532A3E0F533A30C
:10123C00E0F53412288D752FFF75301F7531FF7551
:10124C0032FF75332075340B7BFF7A1F79D8122847
:10125C008D7BFF7A20791412288D7BFF7A20797A86
:10126C0012288D7BFF7A2079A79077C3E0F52FA306
:10127C00E0F530A3E0F531A3E0F53212288D7BFFC9
:10128C007A2079D19077CCE0F52FA3E0F530A3E06C
:10129C00F531A3E0F53212288D7BFF7A2079FF908F
:1012AC0077D0E0F52FA3E0F530A3E0F531A3E0F51E
:1012BC003212288D7BFF7A21792D9077B9E0F52FAA
:1012CC00A3E0F530A3E0F531A3E0F53212288D7BD5
:1012DC00FF7A2179509077B5E0F52FA3E0F530A394
:1012EC00E0F531A3E0F53212288D7BFF7A21796D80
:1012FC009077D4E0F52F12288D7BFF7A2179971205
:10130C00288D7BFF7A2179C0A21EE433F52F122899
:10131C008D7BFF7A2179F0907AFFE0F52F12288DE2
:10132C007BFF7A22791D907B09E0F52F12288D7BAB
:10133C00FF7A227950907732E0F52F12288D7BFFBF
:10134C007A22797EA211E433F52F12288D7BFF7A55
:10135C002279AA907AF9E0F52FA3E0F530A3E0F515
:10136C0031A3E0F532A3E0F533A3E0F53412288D78
:10137C00123F907BFF7A2279F512288D229077F418
:10138C00E0644C70527E227FFB1245129077FCE099
:10139C00F527A3E0F528E4F5297D03AF28AE271245
:1013AC0045F37E237F36124512AE27AF28E4FB7D32
:1013BC00101246CD7E237F3912451274102528F564
:1013CC0028E43527F5270529E529C3941040CA7E62
:1013DC00237F39124512229077F4E0646C705CF52F
:1013EC002B7E237F3B124512E4F52AAF2B7E007D2A
:1013FC00031245F37E237F36124512E4F529A82B00
:10140C00E6FF74FE2529F582E43477F583EFF005C9
:10141C002B0529E529B410E67E777FFEE4FB7D10D1
:10142C001246CD7E237F39124512052AE52AC39434
:10143C000840B87E237F39124512229077F4E0647D
:10144C004B7061F52974E62529F582E43477F58330
:10145C00E0603274E62529F582E43477F583E0F414
:10146C00602374E62529F582E43477F583E0FF7474
:10147C00FC2529F582E43477F583E0B507100529BE
:10148C00E529B408C09075807432F0021945907744
:10149C00F47421F0301A030219457E237F7612452D
:1014AC00120219459077F4E0B4521A201A077E23E1
:1014BC007F7E1245129077F47472F07E777FF47D04
:1014CC0008124B06229077F4E064497045201A0705
:1014DC007E237F891245129077FCE0F527A3E0F577
:1014EC0028E4F529852882852783E0FF74FE2529C9
:1014FC00F582E43477F583EFF00528E528700205D2
:10150C00270529E529B480DC7E777FF47D8A124B90
:10151C0006229077F4E064437079A3E0645270463D
:10152C00201A077E237F911245129077FCE0F52755
:10153C00A3E0F528E4F529852882852783E493FF29
:10154C0074FE2529F582E43477F583EFF00528E560
:10155C0028700205270529E529B480DB7E777FF406
:10156C007D8A124B06229077F5E0645760030219CE
:10157C004E9077FCE0F527A3E0F52874FE2529F5BD
:10158C0082E43477AD82FC7B80AF28AE271251EF1A
:10159C000219459077F4E0644460030216309077AA
:1015AC00FCE0FF64447003021945EFB4310CC21A1D
:1015BC007E237F9A1245120219459077FCE0B430D5
:1015CC000CD21A7E237FA61245120219459077FC85
:1015DC00E0B4320CD21B7E237FB3124512021945A4
:1015EC009077FCE0B4330CC21B7E237FC1124512F2
:1015FC000219459077FCE0B4340CD21C7E237FD0CA
:10160C001245120219459077FCE0B4350CC21C7ED1
:10161C00237FDD1245120219459077FCE0FF120082
:10162C001E021945907580E07013201A077E237FE7
:10163C00EB1245129077F47421F0021945907580E5
:10164C007432F09077F4E0FFB45104C2AF80FEEF37
:10165C0064577045201A077E237FF9124512907744
:10166C00FDE09077B0F0E4F5299077B0E0FFE52944
:10167C00C39F400302194574FE2529F582E4347793
:10168C00F583E0FF9077FCE02529242BF582E434E8
:10169C0076F583EFF0052980D09077F4E064536001
:1016AC0003021753201A077E247F041245129077E9
:1016BC00BDE0FF907634E06F703C9077BEE0FF9019
:1016CC007635E06F70309077BFE0FF907636E0B5FE
:1016DC0007249077C0E0FF907637E0B50718907735
:1016EC00C1E0FF907638E0B5070C9077C2E0FF9030
:1016FC007639E06F60169077F47421F0301A03029B
:10170C0019457E247F13124512021945E4F529E48C
:10171C00F50DAF29FE742B2529F582E43476F5837B
:10172C00E0FD1253610529E529C394FE40E1C2AFE7
:10173C00E4907FF0F0A3F0907FFD74AAF0A374FF07
:10174C00F0A37455F080FE9077F4E0644F704C90E9
:10175C0077FCE0F527A3E0F528E5284527700A205B
:10176C001A077E247F1C124512201A077E247F2321
:10177C00124512E4F52974FE2529F582E43477F537
:10178C0083E0852882852783F00528E528700205EB
:10179C00270529E529B480DE0219459077F4E0FF8E
:1017AC00B445219077FCE0FDA3E0907FF0CDF0A351
:1017BC00EDF0C2AF907FFD74AAF0A374FFF0A37498
:1017CC0055F080FEEF646560030219459077FCE0EC
:1017DC00FFA3E0907FF0CFF0A3EFF0E4F527F5281E
:1017EC00D3907FF1E09528907FF0E095274020E49E
:1017FC00F50D2528FFE5273401FE852882852783F2
:10180C00E0FD1253610528E5287002052780D17E82
:10181C00247F251249FDEF4E60201200039077C300
:10182C00EFF01200039077C4EFF01200039077C52D
:10183C00EFF01200039077C6EFF07E247F2B124955
:10184C00FDEF4E60201200039077CCEFF0120003F6
:10185C009077CDEFF01200039077CEEFF0120003EB
:10186C009077CFEFF07E247F311249FDEF4E602050
:10187C001200039077D0EFF01200039077D1EFF0C5
:10188C001200039077D2EFF01200039077D3EFF0B1
:10189C007E247F371249FDEF4E60201200039077B3
:1018AC00B9EFF01200039077BAEFF01200039077C3
:1018BC00BBEFF01200039077BCEFF07E247F3D125B
:1018CC0049FDEF4E60201200039077B5EFF0120047
:1018DC00039077B6EFF01200039077B7EFF0120099
:1018EC00039077B8EFF07E247F431249FDEF4E60F2
:1018FC0008124FE69077D4EFF0E4F529E4F50DE506
:10190C00292401FFE433FE74B52529F582E43477EC
:10191C00F583E0FD1253610529E529C3944340DCAE
:10192C00C2AFE4907FF0F0A3F0907FFD74AAF0A317
:10193C0074FFF0A37455F080FE7E777FF47D08125F
:02194C004B0648
:01194E002276
:1051B700AE07EEC39430400BEED394395005EE247E
:1051C700D0FF22EEC39461400BEED394665005EEF8
:1051D70024A9FF22EEC39441400BEED39446500519
:0851E700EE24C9FF22AF0622ED
:1053470090772BE004F0700690772AE004F09077CE
:0A5357002AE0FEA3E0FF12532B2210
:100003001253471251B7EFC454F0FEC006125347C0
:080013001251B7D0E02FFF22CB
:104FE600E4907C37F0125347907C38EFF0C394304E
:104FF6004018E0FFD394395011907C37E02483F5B4
:1050060082E43475F583EFF08011907C37E02483D9
:10501600F582E43475F583E4F0800C907C37E00487
:10502600F0E0D3940840BE752F007530007531004E
:0C503600E4F5327B017A757983123B119E
:01504200224B
:0449FD008E2C8F2D40
:104A010090772AE4F0A374FFF0125347EF606EF43D
:104A1100606B852D82852C83E493B507EC752E019F
:104A2100E52D252EF582E4352CF583E49360259060
:104A3100772BE0252EFF90772AE03400FE12532BCE
:104A4100E52D252EF582E4352CF583E493B5070495
:104A5100052E80CCE52D252EF582E4352CF583E459
:104A61009370A6E52E24FFFFE434FFFE90772BE040
:104A71002FF090772AE03EF07E007F0122E4FEFFD6
:014A81002212
:10442C007E247F741249FDEF4E70037F01227E249F
:10443C007F771249FDEF4E600C125347EF24D024C6
:10444C00FF921E8002D21E7E247F7D1249FDEF4E0C
:10445C00600C125347EF24D0907AFFF08005E49063
:10446C007AFFF07E247F831249FDEF4E600C1253CD
:10447C0047EF24D0907B09F08005E4907B09F07E17
:10448C00247F891249FDEF4E600C125347EF24D064
:10449C00907732F08005E4907732F07E247F8F1293
:1044AC0049FDEF4E600C125347EF24D024FF9211BC
:1044BC008002C2119077BD63A201907AF963A201C8
:1044CC007F0612388B30113B7E247F951249FDEF0D
:1044DC004E6030120003907AF9EFF0120003907ADC
:1044EC00FAEFF0120003907AFBEFF0120003907ACF
:1044FC00FCEFF0120003907AFDEFF0120003907ABB
:06450C00FEEFF07F00222B
:1035BD00C211E4907B09F0D21EC214907AFFF090F4
:1035CD007732F09077BD63A201907AF963A2017F03
:1035DD000612388BE4F527E52775F003A4249BF537
:1035ED0082E43424F583E493FB740193FA7402931B
:1035FD00F91224B370030237AFE4F528F529FD74F1
:10360D00AB2DF582E43475F583E0FF70030237AA24
:10361D00E52775F003A4249BF582E43424F583E4B7
:10362D0093FB740193FA740293F9852882758300D4
:10363D001224CCFEEFB5060875290105280237A620
:10364D00E52970030237A6EE60030237A1E52724B2
:10365D00FE602814700302378914700302378D142D
:10366D007003023795147003023799240560030225
:10367D0037AA907B097401F00237AAD21174AB2DD1
:10368D00F582E43475F583E0FF642D70030237AAEB
:10369D001251B7EFC454F0FC74AC2DF582E43475BF
:1036AD00F583E0FF1251B7EF2C907AF9F074AD2D40
:1036BD00F582E43475F583E0FF1251B7EFC454F091
:1036CD00FC74AE2DF582E43475F583E0FF1251B72D
:1036DD00EF2C907AFAF074AF2DF582E43475F58302
:1036ED00E0FF1251B7EFC454F0FC74B02DF582E435
:1036FD003475F583E0FF1251B7EF2C907AFBF0741F
:10370D00B12DF582E43475F583E0FF1251B7EFC4A6
:10371D0054F0FC74B22DF582E43475F583E0FF129C
:10372D0051B7EF2C907AFCF074B32DF582E434751B
:10373D00F583E0FF1251B7EFC454F0FC74B42DF5CE
:10374D0082E43475F583E0FF1251B7EF2C907AFDCA
:10375D00F074B52DF582E43475F583E0FF1251B7A1
:10376D00EFC454F0FC74B62DF582E43475F583E0A6
:10377D00FF1251B7EF2C907AFEF08021D214801DEC
:10378D00907AFF7401F08015C21E8011907732740B
:10379D0001F08009E4F529F5280D02360C05270204
:0237AD0035E401
:0137AF0022F7
:1050F4009079F5E0C3947C503D9079F5E0FE04F09E
:1051040074332EF582E43477F583EFF0BF0A2790E9
:1051140079F5E0FF04F074332FF582E43477F583F6
:10512400E4F09079F5E0FF124B889079F57408F07B
:07513400907734E004F02243
:105043009080007480F09077B563A201F583F582B8
:1050530063A2017F0812388B9077BD63A201908011
:105063008863A2017F0A12388B908092E4F0A374C4
:1050730032F0A37401F09077C7E0FF9080B1F09015
:1050830080E1EFF09080957455F0A3F09080007468
:0950930001F09080097470F02214
:104CFF00908009E04410F09080A0E0706C9080A14B
:104D0F007482F09080A874FFF0A3F0A3F0A3F07F5B
:104D1F00039080AEEFF07FCBA3EFF07F039080ACDA
:104D2F00EFF0A374CBF09080007402F0907C291206
:104D3F00260800000000907C29E0908040F0907CD5
:104D4F002AE0908041F0907C2BE0908042F0907CA4
:104D5F002CE0908043F0A3E4F0A3F0A3F0A3F09035
:094D6F008018F0A3F0A3F0A3F0FA
:014D78002218
:104EC100908009E04440F09080D17482F09077C8DE
:104ED100E0FF9080DEF09077C9E0FF9080DFF090F6
:104EE10080027402F0907C2D1226080000000090D0
:104EF1007C2DE0908058F0907C2EE0908059F090CD
:104F01007C2FE090805AF0907C30E090805BF0A3A1
:104F1100E4F0A3F0A3F0A3F0908030F0A3F0A3F0AD
:024F2100A3F0FB
:014F2300226B
:104D7900908009E04420F09080B8E0706C9080B990
:104D89007482F07F039080C6EFF07FCDA3EFF07FB0
:104D9900039080C4EFF0A374CDF09080C074FFF04D
:104DA900A3F0A3F0A3F09080017402F0907C31127B
:104DB900260800000000907C2DE090804CF0907C4B
:104DC9002EE090804DF0907C2FE090804EF0907C0A
:104DD90030E090804FF0A3E4F0A3F0A3F0A3F090AB
:094DE9008024F0A3F0A3F0A3F074
:014DF200229E
:104A82008C278D28A907EAFDE975F018A424ACFF4C
:104A9200E5F034808F82F583EDF0EBFDE975F018D7
:104AA200A4FFAEF024ACFBEE34808B82F583A3ED41
:104AB200F08528828C83E0FDEF24A8FFEE3480FE8F
:104AC2008F82F583EDF08528828C83A3E08F828E1E
:104AD20083A3F0852882852783A3A3E0FDE975F0EF
:104AE20018A424A8FFE5F03480FE8F82F583A3A3E7
:104AF200EDF08528828C83A3A3A3E08F828E83A30B
:044B0200A3A3F02257
:064B06008D2CAB07AA068E
:104B0C00907C29E0FCA3E0FDA3E0FEA3E0F5308E51
:104B1C002F8D2E8C2DAE02AF038E838F8263A2015C
:104B2C00E52F540744C0F58385308263A201AF2C76
:104B3C001238F4908000E020E5F9E4FCFDFEE5304D
:104B4C00252CF530EE352FF52FED352EF52EEC35D9
:104B5C002DF52D908040E52DF0A3E52EF0A3E52F4B
:104B6C00F0A3E530F09080007420F0AF30AE2FADA4
:0B4B7C002EAC2D907C291225FCAF2CE4
:014B8700220B
:064C84008D27AB07AA0614
:104C8A00907C2DE0FCA3E0FDA3E0FEA3E0F52B8ED3
:104C9A002A8D298C28AE02AF038E838F8263A201EC
:104CAA00E52A540744D0F583852B8263A201AF27F6
:104CBA001238F4E4FCFDFEE52B2527F52BEE352A08
:104CCA00F52AED3529F529EC3528F528908058E59F
:104CDA0028F0A3E529F0A3E52AF0A3E52BF09080BC
:104CEA00027420F0AF2BAE2AAD29AC28907C2D128D
:044CFA0025FCAF27BF
:014CFE002293
:0247A1008F285F
:1047A300908001E030E5037F0022907C31E0FCA3A0
:1047B300E0FDA3E0FEA3E0F52C8E2B8D2A8C29903F
:1047C3007AF963A201E52B540744C8F583852C824B
:1047D30063A2017F0612390AE52C2406F52CE43581
:1047E3002BF52BE4352AF52AE43529F5299079F7B9
:1047F30063A201E52B540744C8F583852C8263A289
:1048030001AF2812390AE4FCFDFEE52C2528F52C1E
:10481300EE352BF52BED352AF52AEC3529F52990C4
:10482300804CE529F0A3E52AF0A3E52BF0A3E52CC2
:10483300F09080017420F0AF2CAE2BAD2AAC299000
:074843007C311225FCAF28B7
:01484A00224B
:104328009081E0E0F52705270527052705270527BC
:1043380005270527052705270527908010E0F52A7A
:10434800A3E0F52BA3E0F52CA3E0F52D9081E1E0A7
:10435800F527052705270527052705270527052705
:10436800052705270527908014E0F52EA3E0F52FF3
:10437800A3E0F530A3E0F531E530B52C08E531B51B
:104388002D037F0022E4F527E530540744E0F58348
:1043980085318263A2019077F463A2017F08123904
:1043A800229077F663A20190772C63A2017F061210
:1043B800388B9077F4E0F528A3E0F529E4F5279009
:1043C80077F4E0702AA3E024F8F527E53054074491
:1043D800E0F58385318274082582F582E43583F51A
:1043E8008363A2019077F463A201AF27123922AE4A
:1043F80028E4FCFDE5312529F531E5303EF530EDC1
:10440800352FF52FEC352EF52E908014E52EF0A3E0
:10441800E52FF0A3E530F0A3E531F090800074407B
:03442800F0AF27CB
:01442B00226E
:103CB5009081E6E0F5270527052705270527052730
:103CC50005270527052705270527908028E0F52ADC
:103CD500A3E0F52BA3E0F52CA3E0F52D9081E7E01B
:103CE500F52705270527052705270527052705277F
:103CF50005270527052790802CE0F52EA3E0F52F55
:103D0500A3E0F530A3E0F531E4F527E530B52C0A5D
:103D1500E531B52D05C218023E0FE530540744F0D4
:103D2500F58385318263A2019077F463A2017F0850
:103D35001239229077F4E0F528A3E0F529E5294525
:103D45002870099080027410F07F0022907B00E0BB
:103D5500FFF4602D9077F6E06F7076907B01E0FFC1
:103D65009077F7E06F706A907B02E0FF9077F8E05C
:103D75006F705E907B03E0FF9077F9E06F602280C3
:103D8500509077F6E0907B00F09077F7E0907B011C
:103D9500F09077F8E0907B02F09077F9E0907B0364
:103DA500F09077F4E0702AA3E024F8F527E5305485
:103DB5000744F0F58385318274082582F582E43560
:103DC50083F58363A2019077F463A201AF271239CB
:103DD50022AE28E4FCFDE5312529F531E5303EF537
:103DE50030ED352FF52FEC352EF52EAF2DAE2CAD54
:103DF5002BAC2AAB31AA30A92FA82ED31225EB4024
:103E0500099080027410F07F002290802CE52EF03E
:103E1500A3E52FF0A3E530F0A3E531F0908002741F
:043E250040F0AF2793
:013E29002276
:103E2A009081E3E0F52705270527052705270527BC
:103E3A000527052705270527052790801CE0F52A71
:103E4A00A3E0F52BA3E0F52CA3E0F52D9081E4E0A7
:103E5A00F527052705270527052705270527052708
:103E6A00052705270527908020E0F52EA3E0F52FEA
:103E7A00A3E0F530A3E0F531E4F527E530B52C0AE7
:103E8A00E531B52D05C219023F75E530540744E8FE
:103E9A00F58385318263A20190748063A2017F0E4B
:103EAA00123938907480E0F528A3E0F529907488D7
:103EBA00E0FFF46045907AF9E0FEEF6E706EA3E0E1
:103ECA00FF907489E06F7064907AFBE0FF90748AC7
:103EDA00E06F7058907AFCE0FF90748BE06F704C42
:103EEA00907AFDE0FF90748CE06F7040907AFEE06B
:103EFA00FF90748DE06F60048032D28D907480E000
:103F0A00702AA3E024F2F527E530540744E8F58344
:103F1A00853182740E2582F582E43583F58363A2A6
:103F2A000190748063A201AF27123938AE28E4FCED
:103F3A00FDE5312529F531E5303EF530ED352FF532
:103F4A002FEC352EF52EAF2DAE2CAD2BAC2AAB3186
:103F5A00AA30A92FA82ED31225EB5006E529452809
:103F6A0070099080017410F07F0022908020E52E65
:103F7A00F0A3E52FF0A3E530F0A3E531F09080013E
:053F8A007440F0AF27B8
:013F8F00220F
:044512008E2C8F2D2F
:10451600907C29E0FCA3E0FDA3E0FEA3E0F5338E4A
:10452600328D318C30E533FFE5325407FEE42FF54A
:104536002FEE34C0F52E852F82F5837423F0052FD8
:10454600E52F7002052E532EC7F582852E83740A39
:10455600F0052FE52F7002052E532EC79077BD6309
:10456600A201852E83852F8263A2017F061238F46D
:104576007406252FF52FE4352EF52E852C83852DF3
:104586008263A201852E83852F8263A2011238D809
:10459600908000E020E5F9E4FCFDFE907C29E0F83F
:1045A600A3E0F9A3E0FAA3E02FFFEE3AFEED39FD12
:1045B600EC38FCEF2408FFE43EFEE43DFDE43CFC61
:1045C600907C291225FC907C29E0908040F0907C1C
:1045D6002AE0908041F0907C2BE0908042F0907C25
:0C45E6002CE0908043F09080007420F0E6
:0145F20022A6
:0646CD008E2C8F2D8D2EB6
:1046D300907C29E0FCA3E0FDA3E0FEA3E0F5348E8B
:1046E300338D328C31E534FFE5335407FEE42FF587
:1046F30030EE34C0F52F853082F5837423F0053016
:10470300E5307002052F532FC7F582852F83EBF019
:104713000530E5307002052F532FC79077BD63A294
:1047230001852F8385308263A2017F061238F474DA
:10473300062530F530E4352FF52F852C83852D8222
:1047430063A201852F8385308263A201AF2E1238C5
:10475300F4908000E020E5F97408252EF52EFFE49F
:10476300FCFDFEE5342FF534EE3533F533ED35320C
:10477300F532EC3531F531908040E531F0A3E53287
:10478300F0A3E533F0A3E534F09080007420F0AF9C
:0D47930034AE33AD32AC31907C291225FCE0
:0147A00022F6
:024B88008F405C
:104B8A00907C29E0FCA3E0FDA3E0FEA3E0F5448EBF
:104B9A00438D428C41E544FFE5435407FEE42FFF71
:104BAA00EE34C090773363A201F5838F8263A2014A
:104BBA00AF401238F4908000E020E5F9E4FCFDFEF5
:104BCA00E5442540F544EE3543F543ED3542F542DB
:104BDA00EC3541F541908040E541F0A3E542F0A370
:104BEA00E543F0A3E544F09080007420F0AF44AEB2
:0B4BFA0043AD42AC41907C291225FC29
:014C0500228C
:0645F3008E2C8F2DAB059C
:1045F900907C29E0FCA3E0FDA3E0FEA3E0F5338E67
:10460900328D318C30E533FFE5325407FEE42FF566
:104619002FEE34C0F52E852F82F5837423F0052FF4
:10462900E52F7002052E532EC7F582852E83EBF0F8
:10463900052FE52F7002052E9077BD63A201852E07
:1046490083852F8263A2017F061238F47406252F11
:10465900F52FE4352EF52E532EC7E52C852F8285AF
:104669002E83F0052FE52F7002052E532EC7F582F4
:10467900852E83E52DF0052FE52F7002052E532E8B
:10468900C7908000E020E5F9E533240AF533E435E5
:1046990032F532E43531F531E43530F5309080408A
:1046A900E530F0A3E531F0A3E532F0A3E533F0906E
:1046B90080007420F0AF33AE32AD31AC30907C293C
:0346C9001225FCBB
:0146CC0022CB
:10532B00E5D220E0FBC2AF438E2075D2028F828E76
:0B533B0083E0FFE4F5D2538EDFD2AF19
:015346002244
:10536100E5D220E0FBC2AF43D2028F828E83EDF003
:0953710075D25063D250D2AF2274
:104C0600E4FDED2401FFE433FE12532B74B52DF5BC
:104C160082E43477F583EFF00DBD3FE6E4FDED2445
:104C26007FFFE433FE12532B74AB2DF582E434750B
:104C3600F583EFF074AB2DF582E43475F583E070FF
:104C46001B74AB2DF582E43475F5837420F074ACD7
:104C56002DF582E43475F583E4F080040DBD80BE45
:104C6600E490762AF0FDEDFF7E0012532B742B2D77
:0D4C7600F582E43476F583EFF00DBDFEE924
:014C8300220E
:0251EF008B2C07
:1051F100A2AF921FC2AF85A22D53A2FE8E838F82D2
:1052010005A28C838D827409123950E52C53A2FEBC
:1052110043A22012395253A2DF852DA2A21F92AFC1
:01522100FF8D
:015222002269
:10530E00A2AF921FC2AF8C838D82EF12395043A28F
:0C531E002012395253A2DFA21F92AFFFF1
:01532A002260
:0252A2008F2754
:1052A400A2AF921FC2AFE4F5838D82740612395007
:1052B400E52743A22012395253A2DFA21F92AF7FE7
:0152C40001E8
:0152C50022C6
:0252C6008F2730
:1052C800A2AF921FC2AFE4F5838D82740A123950DF
:1052D800E52743A22012395253A2DFA21F92AF7FC3
:0152E80001C4
:0152E90022A2
:1037B000A907E7FFA805EF93C3966008403B74FC98
:1037C0002FFF80F00F08EF93C3966008402B74FB27
:1037D0002FFF80E00F08EF93C3966008401B74FA38
:1037E0002FFF80D00F08EF93D3966008400B74F939
:1037F0002FFF80C01F1F1F1F1FEF54FEF80303F78A
:10380000E893FC08E893FD08E893FE08E893FF229C
:1038100009E993C39D6008402974FB29F980F109E7
:10382000E993C39E6008401A74FA29F980E209E915
:1038300093D39F6008400B74F929F980D3191919A3
:103840001919E9C313C313FF22740093F8ECC3984A
:103850004024701F740193F8EDC3984019701474DC
:0E3860000293F8EEC398400E7009740393F8BB
:10386E00EFC39840037F00227F0122EDF8E6F008B7
:10387E00A3DFFA22EDF8E0F608A3DFFA22E0A36355
:10388E00A201F0A363A201DFF475A20022E0A363FC
:10389E00A201F0A363A201E0A363A201F0A363A2BD
:1038AE0001E463A201F0A363A201DFE175A200228D
:1038BE00E0A363A2016DFE936CFDEE058393FC15F0
:1038CE008363A201DFEA75A200227F00E493A36363
:1038DE00A201F00F600CA3E583C2E3F58363A2019E
:1038EE0080EA75A20022E0A363A201F0A3E583C2E1
:1038FE00E3F58363A201DFEE75A20022E0A363A2CB
:10390E0001F0A3E583C2E4D2E3F58363A201DFEC09
:10391E0075A20022E583C2E3F583E0A363A201F062
:10392E00A363A201DFEE75A20022E583C2E4D2E317
:10393E00F583E0A363A201F0A363A201DFEC75A2FD
:10394E000022F922C002C004C00612FFF0D006D039
:04395E0004D002226D
:104DF3000A536572763A00205544502054696D6514
:104E03004750530A00200A444154414752414D3A06
:104E130020002043414E2054696D654750530A00DA
:104E230020547261737353656E644552520A0020B5
:104E33005265496E69742043414E0A002043414E36
:104E4300283029203E20544F210A00205455203079
:094E53000A0020545520310A0028
:03001E00E4FF22DA
:10525600C28DC2AF438901C28C907B1FE0FF7007ED
:10526600F58A758CEE800AEFB40A06E4F58A758C29
:0652760070D28CD2AF22C1
:10522300C28DC2AF438901C28C907B1FE0FF701413
:10523300302C09F58A758CDCC22C8012758A667550
:105243008CFC800AEFB40A06E4F58A758CDCD28CF8
:03525300D2AF22B5
:10527C00C22D907B1FE0C394645006124E5C1252F8
:10528C0056120022D22BE4F570907C27F0F55EF5D7
:06529C0074C22CF5722221
:10513B00EF24FCF527201A127E4D7FF31245127EC9
:10514B00777FF8E4FBAD271246CD9077F7E0B41FDD
:10515B0003D22D229077F863A201907BA763A20163
:0D516B00AF2712388B85275EE4F56FC2294F
:015178002214
:0F539100D3EF6480948E5006E57470028F7422FF
:102B8700208D03022C8DC28C202B03022D8AE57425
:102B970060519074807D60FF123882E56064017037
:102BA7001E907488E0B4FF0ED22E201A127E4D7F3D
:102BB700FA1245128009302E06E4F574022D8A12A6
:102BC7005256124F24201A077E4E7F0812451220B4
:102BD7001A0B7E747F80E4FBAD741246CDE4F57466
:102BE700022D8AE55E605C74AB256FF582E4347B69
:102BF700F583E02405F527D3940E4008E4F55ED26B
:102C070029022D8A74A7256FF582E4347BF5837D2D
:102C170060AF27123882E527256FF56FE56030E74B
:102C270002D22CE560B40103202E06125256124F31
:102C370024E56FC3955E5003022D8AE4F55ED22921
:102C4700022D8AE5716023907B0B7D60FF1238822D
:102C5700E560B40109302E06E4F571022D8A12529F
:102C670056124F24E4F571022D8A200016E573C32E
:102C77009464400320130C907B1FE0C394645003BB
:102C8700124F861252561240DF8F27EF7003022D24
:102C97008A125223E4F572E560B4010CD22E201A91
:102CA700077E4E7F15124512E573C3946E400302EB
:102CB7002D61201303022D61302D75E5606442708C
:102CC7006FE5647032E562C454F0FFE563C4540FE6
:102CD7002FF560E563C454F0F5617562087420252B
:102CE70073F582E4347BF58374032573F5737D6094
:102CF7007F03123879806374202573F582E4347B6F
:102D0700F583E5272573F5737D60AF271238793092
:102D17001C48C3E5739527FFE49400FE74202FF544
:102D270082747B3EAF82FEE4FBAD271246CD802A3C
:102D3700E560B4420DE563B40208907732E06401C0
:102D4700601874202573F582E4347BF583E5272525
:102D570073F5737D60AF27123879301121E5602054
:102D6700E71C9079F77D60AF27123879AF271247B4
:102D7700A1EF700A201A077E4E7F23124512AF2754
:102D8700124213301D1A301015907B1FE0C3946454
:102D9700500C0572E57294F04004C2AF80FEC21D6C
:102DA700201203022ED2906001E004F070069060BA
:102DB70000E004F0E5566021906195E07002A3E021
:102DC7006017906196E024FFF0906195E034FFF082
:102DD700E07002A3E07002D203E5706031D3940182
:102DE700400415708028907C27E004F0E0D394031A
:102DF700400D201A077E4E7F3212451212527C2058
:102E07001A077E4E7F3F124512E4F570D22B302A07
:102E170043E571703F907B0B04F0A37408F0A37433
:102E270080F0A37401F0A37406F0907BA2E0907B7E
:102E370010F0907BA3E0907B11F0907BA4E0907B57
:102E470012F0907BA5E0907B13F0E4A3F0A3F0755C
:102E5700710BC22A302872907BA0E07035E5717043
:102E670031907B0B7442F0A37408F0907BA1E09043
:102E77007B0DF0907BA6E0907B0EF0A37401F075BC
:102E87007106201A077E4E7F4E124512907BA0E0F6
:102E970004F0907BA0E06402702FE571702B907BAB
:102EA7000B7402F0A37408F0907BA1E0907B0DF007
:102EB700A3F0A37401F0757106201A077E4E7F55A3
:0E2EC700124512907BA0E004F0C2121208C463
:012ED50022DA
:10517900E5736037E49078F4F0A3E573F0907AF87A
:10518900E09078F6F0302D06A3741FF08006907831
:10519900F77419F0907B2063A2019078F863A2015B
:0E51A900AF7312388BE4F5737F01227F002272
:0B53A000302905C2297F01227F002276
:0100210022BC
:0653C500E4F573F55E2221
:0A53AB00E4907583F0A3F0A3F02254
:1052EA002043616E457247495400200A00204361F9
:1052FA006E457272434821000A000A2052657145C0
:04530A00727221009A
:1040DF00E59B541F6020201A1A7E527FEA12451268
:1040EF00E59B541FFF7E007D031245F37E527FF444
:1040FF00124512E4F59BE5BA30E010E4F5B375B163
:10410F0080F5B2D22BF570907C27F0E5CFF47003D9
:10411F00024210752901E4F528E5CFF45529700303
:10412F000241FEE528C454F0F5B1E5B2547F642096
:10413F0060030241CFE5B3540FF56485BC60E5BD64
:10414F00541FFF131313541FFFE5BD54E044184FC2
:10415F00F561E5BDC43354E0FFE5BE131313541FDF
:10416F004FF562E5BEC43354E0FFE5BF131313549C
:10417F001F4FF56385A36585A36685A36785A36830
:10418F0085A36985A36A85A36B85A36CE4F5B2202B
:10419F00000CE560547EB5600575B350800375B3B0
:1041AF00D0E564700AE560547EB560037F0022306D
:1041BF000008E56030E7037F0022E5642405FF2255
:1041CF00E5B2549F6023201A207E527FF7124512CA
:1041DF00AFB27E007D031245F3AFB37E007D0312B5
:1041EF0045F37E537F02124512E4F5B275B3D0E565
:1041FF002925E0F5290528E528C394085003024135
:03420F00287F0005
:014212002289
:104F2400907B1FE0C39464505675B180E4F5B3F5EB
:104F3400B28560BCE562C4135407FFE56154E04FD9
:104F4400F5BDE56233333354F8FFE563C413540706
:104F54004FF5BEE56333333354F8F5BF8565A38558
:104F640066A38567A38568A38569A3856AA3856B02
:104F7400A3856CA3E564540F2450F5B375700AC27D
:024F84002B22DE
:104F860075B190E5B220E613201A107E537F041205
:104F96004512AFB27E007D031245F3E4F5B3F5B2D8
:104FA600749C250FF582E43461F583E0F5BCE4F5E5
:104FB600BD749D250FF582E43461F583E0FF33333C
:104FC6003354F8F5BE75BF78050F050F749C250F91
:104FD600F582E43461F583E07002F50F75B3502273
:0953B500EF6003C29622D2962299
:104E5C0043AB01C2E8C2EAE4FFEFC454F0F5B1C3BE
:104E6C00EF64809488500575B3D08003E4F5B3E407
:104E7C00F5B2F5BCF5BDF5BEF5BFF5C4F5C5F5C687
:104E8C00F5C7F5A3F5A3F5A3F5A3F5A3F5A3F5A332
:104E9C00F5A30FBF0EC3907B1FE0FF25E0F5B475A3
:104EAC00B50C75B66C75A11275AB0275C13E75C3A8
:044EBC00FF75C203B9
:014EC00022CF
:100026005452414E5A004D415842005254530044D6
:10003600454C4159004E4F4B5654004B5000424FD1
:100046004F540043414E004E4557504B54004154C7
:10005600004443440043414E4D4F4E0054454C3AF4
:10006600004C434C004454420054524300003E2A84
:100076002C312CCFE0F0E0ECE5F2F0FB20F3EFF0D2
:10008600E0E2EBFFFEF9E5E3EE20EAEEEDF2F0EE5C
:10009600EBEBE5F0E020CACF20C8F1E5F2FC0A0060
:1000A6003E4C2C6B30312C25732C43EAEEF0EEF1EE
:1000B600F2FC20EDE020F8E8EDE52043414E2C303F
:1000C600202D20353030EAE1283530EC292C31203E
:1000D6002D203530EAE128353030EC290A00302071
:1000E6002D20353030EAE1283530EC290031202D3D
:1000F600203530EAE128353030EC29003E532C6BB0
:1001060030322C2562752CCCE0EAF12E20E0E4F0AA
:10011600E5F120E1EBEEEAE020D2D128302D3829B6
:100126000A003E532C6B30332C2562752CCCE0EA4A
:10013600F12E20E0E4F0E5F120E1EBEEEAE020D25A
:10014600C8D228302D38290A003E532C6B30342C67
:100156002562752CCCE0EAF12E20E0E4F0E5F120F2
:10016600E1EBEEEAE020D2D328302D38290A003E12
:10017600422C6330312C2562752CC2F2EEF0E8F782
:10018600EDFBE920EAEEEDF2F0EEEBEBE5F020ED2B
:10019600E020F8E8EDE50A003E2A2C312CCFE0F00D
:1001A600E0ECE5F2F0FB20EFF0EEF2EEEAEEEBE04B
:1001B60020C8F1E5F2FC20EFEE20EFEEF0F2F3209E
:1001C60052533233320A003E4C2C6B30352C256CA0
:1001D600752CD1EAEEF0EEF1F2FC20EEE1ECE5ED65
:1001E600E020EDE020EFEEF0F2F32C3130302C324F
:1001F60030302C3330302C3630302C313230302CFD
:10020600323430302C343830302C393630302C31D2
:10021600393230302C33383430302C3537363030B4
:100226002C3131353230300A003E532C6B30362CAF
:100236002562752CCDEEECE5F020CACF20E4EBFF6D
:1002460020ECE0E3E8F1F2F0E0EBE8202830202DA6
:1002560020F0E0E4E8E0EBFCEDFBE920EAE0EDE08D
:10026600EB290A003E422C6B30372C2562752CCECA
:10027600E1ECE5ED20E1E5E720EAE2E8F2E0EDF683
:10028600E8E90A003E422C6B30382C2562752CC4F6
:10029600E5EBE0F2FC20E7E0EFF0EEF120F1EEE531
:1002A600E4E8EDE5EDE8FF0A003E422C6B30392C20
:1002B6002562752CCDE520EFE5F0E5E4E0E2E0F21D
:1002C600FC20E4E8E0E3EDEEF1F2E8EAF30A003EB2
:1002D600422C6B31302C2562752CCFE5F0E5E7E03A
:1002E600E3F0F3E7EAE020EFF0E820EEF2F1F3F2D4
:1002F600F1F2E2E8E820EEE1ECE5EDE0203220EC78
:10030600E8ED2E0A003E2A2C312CCFE0F0E0ECE599
:10031600F2F0FB20EEE1ECE5EDE020F120E8F1EF74
:10032600EEEBFCE7EEE2E0EDE8E5EC20EAEEECECE5
:10033600F3F2E8F0F3E5ECEEE920EBE8EDE8E80AA5
:10034600003E422C6B31312C2562752CCEE1ECE55A
:10035600ED20F7E5F0E5E720EAEEECECF3F2E8F065
:10036600F3E5ECF3FE20EBE8EDE8FE20F1E2FFE733
:10037600E80A003E532C6B31322C2D2CCDEEECE5E9
:10038600F020F2E5EBE5F4EEEDE020E4EBFF20F102
:10039600EEE5E4E8EDE5EDE8FF0A003E532C6B31AF
:1003A600322C25732CCDEEECE5F020F2E5EBE5F4EE
:1003B600EEEDE020E4EBFF20F1EEE5E4E8EDE5ED1F
:1003C600E8FF0A003E532C6B31332C2562752CCA8C
:1003D600EEEBE8F7E5F1F2E2EE20EFEEE2F2EEF018
:1003E600EEE220F1EEE5E4E8EDE5EDE8FF0A003E99
:1003F600422C6B31342C2562752CCAEEEDF2F0EEF0
:10040600EBFC20F1EEE5E4E8EDE5EDE8FF20EFEEAC
:1004160020F1E8E3EDE0EBF320ECEEE4E5ECE020A0
:1004260028444344290A003C21003C6B30313D00FE
:100436003C6B30323D003C6B30333D003C6B30341E
:100446003D003C6330313D003C6B30353D003C6B3C
:1004560030363D003C6B30373D003C6B30383D005C
:100466003C6B30393D003C6B31303D003C6B3131EB
:100476003D003C6B31323D003C6B31333D003C6B03
:1004860031343D000A4173796E634F55543A004446
:1004960043445F4F4646210A00446973636F6E6E9C
:1004A6006563746564210A004D4F44454D5F4F4BAB
:1004B600210A004D4F44454D5F434F4E4E45435430
:1004C600210A004D4F44454D5F4C495354454E213A
:1004D6000A004D4F44454D5F4552524F52210A0086
:1004E6004D4F44454D5F434F4E4E4543545F464145
:1004F600494C555245210A004D4F44454D5F4449EC
:1005060053434F4E4E4543544544210A00525453DB
:100516000A004D6F64656D20696E69740A00CDE549
:10052600F220EEF2E2E5F2E0210A004469616C692C
:100536006E670A000D00CEF820E4EBE8EDFB210A19
:10054600000ACDE5F220CAE2E8F2E0EDF6E8E8219D
:10055600000A436F6E66205265712100CCEEE4E519
:10056600EC20E220F5EE2DF0E5E6E8ECE5210A00C8
:10057600C1F0E0EAF3E5EC210A000A4352432045C4
:1005860052523A20000A494E3A000A4173796E6384
:10059600494E3A00436F6E66205265616479210ABE
:1005A60000436F6E6620426C6F636B210A00CFF0CA
:1005B600E8EDFFF2FB20E4E0EDEDFBE520E1E5E709
:1005C60020F1EEE5E4E8EDE5EDE8FF210A000A4456
:1005D6006174613A20003F3F3F0A000089129B2464
:1005E600AD36BF48C15AD36CE57EF78108931AA58C
:1005F6002CB73EC940DB52ED64FF76028B1099267C
:10060600AF34BD4AC358D16EE77CF5830A9118A76B
:100616002EB53CCB42D950EF66FD74048D169F2053
:10062600A932BB4CC55ED768E17AF3850C971EA14B
:1006360028B33ACD44DF56E960FB72068F149D223B
:10064600AB30B94EC75CD56AE378F1870E951CA32B
:100656002AB138CF46DD54EB62F97008811A932C23
:10066600A53EB740C952DB64ED76FF89009B12AD0B
:1006760024BF36C148D35AE56CF77E0A8318912EFB
:10068600A73CB542CB50D966EF74FD8B029910AFEB
:1006960026BD34C34AD158E76EF57C0C851E9728D3
:1006A600A13AB344CD56DF60E972FB8D049F16A9CB
:1006B60020BB32C54CD75EE168F37A0E871C952ABB
:1006C600A338B146CF54DD62EB70F98F069D14ABAB
:1006D60022B930C74ED55CE36AF178001123324661
:1006E6005765748C9DAFBECADBE9F81001332256FC
:1006F6004775649C8DBFAEDACBF9E82130021367EB
:10070600764455ADBC8E9FEBFAC8D93120120377DB
:10071600665445BDAC9E8FFBEAD8C942536170044E
:10072600152736CEDFEDFC8899ABBA5243716014BB
:10073600053726DECFFDEC9889BBAA6372405125AA
:10074600340617EFFECCDDA9B88A9B73625041359B
:10075600241607FFEEDCCDB9A89A8B8495A7B6C2FE
:10076600D3E1F008192B3A4E5F6D7C9485B7A6D27B
:10077600C3F1E018093B2A5E4F7D6CA5B48697E36A
:10078600F2C0D129380A1B6F7E4C5DB5A49687F35B
:10079600E2D0C139281A0B7F6E5C4DC6D7E5F480CE
:1007A60091A3B24A5B69780C1D2F3ED6C7F5E4903B
:1007B60081B3A25A4B79681C0D3F2EE7F6C4D5A12A
:1007C600B082936B7A48592D3C0E1FF7E6D4C5B11B
:1007D600A092837B6A58493D2C1E0F7C2B2B2B7CC9
:1007E6000D6174680D7C61747A0D004F4B0D0A0023
:1007F6000000000000000000000000000000004FA4
:100806004B0D0A0000000000000000000000000080
:10081600000000434F4E4E4543540D0A00000000B1
:10082600000000000000004C495354454E0D0A00DC
:1008360000000000000000000000004552524F5228
:100846000D0A000000000000000000000000004348
:100856004F4E4E454354204641494C5552450D0A8C
:10086600000000444953434F4E4E45435445440D02
:100876000A00000000000000000000000000000068
:100886000000000000000000000000FF0026FF003E
:100896002CFF0031FF0035FF003BFF0041FF004405
:1008A600FF0049FF004DFF0054FF0057FF005BFFAC
:0E08B6000062FF0067FF006BFF006FFF007322
:0300230002319611
:0B319600C0E0C083C082C0D075D0181C
:1031A1002098030232F0C298750B01AF99300103E8
:1031B100023273BF020C906194E4F0D201D2910209
:1031C10032F0200F030232F0900805E493B51F138B
:1031D1009061947401F09061997408F0A37406F001
:1031E100023264900819E493B51F1290619474023D
:1031F100F09061997408F0A3741AF0806690082D1C
:10320100E493B51F129061947403F090619974086E
:10321100F0A3742EF0804C900841E493B51F1290F6
:1032210061947404F09061997408F0A37442F08081
:1032310032900855E493B51F129061947405F09093
:1032410061997408F0A37456F08018900869E493AA
:10325100B51F109061947406F09061997408F0A301
:10326100746AF0906194E070030232F0D201D2915D
:10327100807D906194E0FE6044906199E0FCA3E060
:10328100F5828C83E493B51F2990619AE004F07074
:1032910006906199E004F0BF0A149061CCEEF0A3AE
:1032A100E4F0906194F0C201F54DC2918041054D69
:1032B100803DC291906194E4F0C2018032300A07EE
:1032C100C20A531F0F8019BF0904D20A8021BF030C
:1032D1000F854D58634D80534D80C201C291800FBF
:1032E1007439254DF582E4346FF583EFF0054D20F7
:1032F10099030233AD2002030233AB300973E55465
:10330100B4FF0D7599020554755900D2900233AB83
:10331100E554B54C147599030554906F38E070036A
:103321000233AB7401F00233ABE554D3954C400842
:10333100C202D20FC2908072E5596009F599055415
:10334100755900806574392554F582E43470F5832C
:10335100E0F5596402600BE55964036005E559B471
:103361000905759909804385599905547559008056
:103371003974392554F582E43470F583E0FF70081F
:10338100C202D20FC2908022D290C20FEFB47C0948
:103391000554750832C2028011AF54055474392F97
:0C33A100F582E43470F583E0F599C299E0
:0933AD00D0D0D082D083D0E032F0
:103F90007BFF7A00797412288D907B1FE070147576
:103FA0002FFF7530007531E47BFF7A0079A6122867
:103FB0008D8012752FFF7530007531F37BFF7A000D
:103FC00079A612288D7BFF7A01790290619BE0F53A
:103FD0002F12288D7BFF7A017928906193E0F52FCD
:103FE00012288D7BFF7A01794F906102E0F52F1244
:103FF000288D7BFF7A017975A200E433F52F122812
:104000008D7BFF7A01799E12288D90747AE0FEA351
:10401000E0FFC3E49FFFE49EFEAB07FA3395E0F9AF
:10402000F87F007E8C7D0A7C0012254B8F328E310A
:104030008D308C2F7BFF7A0179CD12288D7BFF7A12
:1040400002792F85562F12288D7BFF7A02796AA27A
:1040500008E433F52F12288D7BFF7A02798AA204B7
:10406000E433F52F12288D7BFF7A0279AFA20BE49F
:1040700033F52F12288D7BFF7A0279D5906F38E0C7
:10408000F52F12288D7BFF7A03790B12288D7BFF89
:104090007A037947A20DE433F52F12288D9061033E
:1040A000E0700B7BFF7A03797912288D8012752FCF
:1040B000017530617531037BFF7A0379A112288D78
:1040C0007BFF7A0379CA907139E0F52F12288D7B36
:0F40D000FF7A0379F5A206E433F52F12288D222B
:103962007E047F2D1249FDEF4E70037F0122E49009
:103972007B1FF07E047F301249FDEF4E601B125315
:10398200478F27E527B43106907B1F740AF0E5279D
:10399200B43206907B1F7464F07E047F361249FDB8
:1039A200EF4E6008124FE690619BEFF07E047F3C81
:1039B2001249FDEF4E6008124FE6906193EFF07EE0
:1039C200047F421249FDEF4E6008124FE6906102F9
:1039D200EFF07E047F481249FDEF4E600D124FE674
:1039E200EC4D4E4F24FF92008002C2007E047F4EB7
:1039F2001249FDEF4E6023124FE6A804A905AA065C
:103A0200AB077F007E8C7D0A7C0012254B1225DDE0
:103A120090747AEEF0A3EFF0800A90747A74FFF05B
:103A2200A374DCF07E047F541249FDEF4E60051250
:103A32004FE68F567E047F5A1249FDEF4E600A12FE
:103A42005347EF24D024FF92087E047F601249FD81
:103A5200EF4E600A125347EF24D024FF92047E04F3
:103A62007F661249FDEF4E600A125347EF24D024BD
:103A7200FF920B7E047F6C1249FDEF4E600A1253D7
:103A820047EF24D0906F38F07E047F721249FDEF29
:103A92004E600A125347EF24D024FF920D7E047F1A
:103AA200781249FDEF4E603CE4F50F1253478F2721
:103AB200E527643C601FE50FC394255018AF0F053E
:103AC2000F74032FF582E43461F583E527F0125376
:103AD200478F2780DB7403250FF582E43461F58379
:103AE200E4F0F50F7E047F7E1249FDEF4E6008126E
:103AF2004FE6907139EFF07E047F841249FDEF4E5C
:0E3B0200600A125347EF24D024FF92067F0082
:013B10002292
:102ED600E4F50F907C37F0907C37E075F003A4247E
:102EE60091F582E43408F583E493FB740193FA7454
:102EF6000293F91224B37003023195E4907C39F001
:102F0600A3F0907C38F0907C38E024ABF582E43472
:102F160075F583E0FF700302318C907C37E075F025
:102F260003A42491F582E43408F583E493FB740149
:102F360093FA740293F9907C39E0F5827583001256
:102F460024CCFEEFB5060F907C3A7401F0907C39E4
:102F5600E004F0023183907C3AE07003023183EEA4
:102F6600600302317A907C37E0B4100040030231EE
:102F76008C902F7EF8282873022FAE022FFB023189
:102F86008C02318C02303802306E02309D02303DA8
:102F960002318C0230A20230F00230F50230FA0221
:102FA600318C02316E023172907C38E024ABF9E448
:102FB6003475FA7B01C0031B8B2F75300075310009
:102FC600E4F532D003123B11907C3B1225FC907C39
:102FD6003BE0F8A3E0F9A3E0FAA3E0FB7F007E8CD8
:102FE6007D0A7C0012254B1225DD90747AEEF0A343
:102FF600EFF002318C907C38E0FD24ABF582E434AE
:1030060075F583E024D090619BF074AC2DF582E4D5
:103016003475F583E024D0906193F0907C38E024F9
:10302600ADF582E43475F583E024D0906102F002B8
:10303600318CD20802318C907C38E024ABF9E43430
:1030460075FA7B01C0031B8B2F753000753100E4C8
:10305600F532D003123B11907C3B1225FC907C3E4E
:10306600E0907B1FF002318C907C38E024ABF9E4D1
:103076003475FA7B01C0031B8B2F75300075310048
:10308600E4F532D003123B11907C3B1225FC907C78
:103096003EE0F55602318CD20402318C907C38E049
:1030A60024ABF9E43475FA7B01C0031B8B2F753012
:1030B60000753100E4F532D003123B11907C3B12CF
:1030C60025FCE4FFFEFDFC907C3BE0F8A3E0F9A3C1
:1030D600E0FAA3E0FBD31225EB4008907C3EE0909B
:1030E6007139F0D20DC20C02318CD20602318CD26B
:1030F6000002318CE4F50F907C38E024ABF582E4D5
:103106003475AF82907C3FF0A3EFF0907C3FE0FEF9
:10311600A3E0F5828E83E0FF6420602AEF6027E556
:103126000FC394255020AE0F050F74032EF582E4CD
:103136003461F583EFF0907C40E004F07006907CFB
:103146003FE004F080C5AF0F050F74032FF582E44E
:103156003461F583740DF07403250FF582E4346150
:10316600F583E4F0F50F801ED20B801A906F387449
:1031760001F08012E4907C3AF0907C39F0907C3833
:0F318600E004F0022F0C907C37E004F0022EDD05
:013195002217
:1033B600E4F54A9061CDF0C207906197F0906F37BF
:1033C6007405F0C202C20FC201C20AE4F554F54CFC
:1033D600F508F54DF50B90747A74FFF0A374F4F0CC
:1033E6009061027402F0906193F090619BF0C20DBF
:1033F600D20CC200907139741EF0E4907B1FF0C2AB
:1034060004C206C205F556C20BC208906F38F0C258
:1034160003906103F0123962EF6003122ED69071A9
:1034260039E004F548E4F50F907C357461F0A37437
:103436009CF090619BE0F50FE50FC394014007E512
:103446000FD394084003E4F50FE50F6028907C3510
:10345600E475F0011224F985F082F58374C4F01541
:103466000F907C35E475F0011224F985F082F5831E
:10347600E50FF080D4906193E0F50FE50FC394015A
:103486004007E50FD394084003E4F50FE50F6028E5
:10349600907C35E475F0011224F985F082F5837489
:1034A600C8F0150F907C35E475F0011224F985F00B
:1034B60082F583E50FF080D4906102E0F50FE50F09
:1034C600C394014007E50FD394084003E4F50FE5E4
:1034D6000F6028907C35E475F0011224F985F0829E
:1034E600F58374C2F0150F907C35E475F001122453
:1034F600F985F082F583E50FF080D4907C35E4758C
:10350600F0011224F985F082F583E4F0907C35759C
:10351600F0011224F985F082F583E4F0F50FF555F4
:1035260075F075E555A4244EF582E5F03468F5830B
:10353600E4F0E55575F00DA4242BF582E43461F52D
:1035460083E4F0F54B75F068E555A4243AF582E579
:10355600F03471F58375F00DE54B122639E4F0056C
:103566004BE54BB407DF0555E555B408B3E4F55D07
:10357600F545F547F549F553F55CF54BF546F55533
:10358600F552C2ADF5C9D2CDD2CCC2C9C2CAF5CDAB
:10359600F5CC90747AE0F5CBA3E0F5CA85CBCD8562
:1035A600CACCD29ED29CD2CAC2ACC298C29975B8B5
:0635B6001075B710D2AC45
:0135BC0022EC
:0100220022BB
:104213008F28300B0EE560B44209E5636402700336
:10422300024327E56154E324DF605624DF6035143D
:10423300603224E360681470030242E914700302DD
:10424300431024E2601E24606003024327E5627585
:10425300F00DA4242BF582E43461F5837D60AF284F
:104263001238792275F00DE549A424F6F582E5F0BC
:10427300346BF5837D60AF28123879054953493F84
:104283002275F00DE545A424CEF582E5F03461F501
:10429300837D60AF28123879054553457F2275F039
:1042A30075E562A4245BF582E5F03468F583E56384
:1042B300543FFF1313543F75F00D1226397D60AF41
:1042C3002812387975F068E562A4243AF582E5F09E
:1042D3003471F583E563543FFF1313543F75F00DB9
:1042E300122639E4F02275F068E562A4243AF582D7
:1042F300E5F03471F583E563543FFF1313543F75C1
:10430300F00D1226397D60AF281238792275F075C9
:10431300E562A4244EF582E5F03468F5837D60AF51
:05432300281238792288
:1048E1008F2B90600263A20190703963A201AF2BFC
:1048F10012388BE4F54EF54F852B5190703963A238
:10490100019005E163A201AF51AE50AD4FAC4E1223
:1049110038BE8F518E508D4F8C4E7439252BF582B8
:10492100E43470F583E54FF0743A252BF582E434D5
:1049310070F583E54EF07439252BF582E43470F57A
:1049410083E0F55AA3E0F55BE52B2402F54C201A30
:10495100127E047F8A1245127E707F39E4FBAD4CD2
:104961001246CD7554FFD202C2992099FDD29922E7
:1008C400301022C210906F38E0600C04F0E0D39432
:1008D400F04004C2AF80FE906198E004F09061CDD6
:1008E400E0600214F0E508B4010CE4F508D202C299
:1008F400992099FDD29930020F906198E0D3941415
:10090400400BC202D20F8005E4906198F0300621BA
:1009140030970E200507907139E004F548D2058020
:100924001030050A201A077E047F95124512C2056D
:1009340022907139E0FFE548D39F403C201A077E9E
:10094400047F9F124512300D15E4906197F0C20C9C
:10095400C209FF1253B59061CD7402F08007E49090
:1009640061CDF0D209E4F54DF558F54AF548C201D8
:10097400906000F0A3F0D20F9061CCE0FF7003020E
:100984000A1224FE601C14602514605114605A1469
:10099400606A24057078201A757E047FAE124512B1
:1009A400806C201A697E047FB91245128060201A77
:1009B400077E047FC9124512300C53E4906197F00E
:1009C400C20CC2099061CDF0F54DF558754A03F596
:1009D40048C201906000F0A3F0D20F8031201A2E9B
:1009E4007E047FD81245128025201A077E047FE6F4
:1009F400124512907139E004F5488012201A077EDE
:100A0400047FFE124512907139E004F54822300C3F
:100A140003020B7B9061CDE06003020B7B200F038C
:100A2400020B7B906197E014603114606E147003C4
:100A3400020B2424036003020B767F011253B5904A
:100A44006197E004F09061CD7401F0301A03020B59
:100A54007B7E057F13124512020B7B201A077E054D
:100A64007F1812451278397C707D017BFF7A0779F3
:100A7400E112270DE4F54DF558F5549061CCF005DD
:100A840048C201D202C2992099FDD299906197E09F
:100A940004F09061CD740AF0020B7B9061CCE0FF0E
:100AA400B403119061977403F005489061CD743CD0
:100AB400F0020B7BEF6401601C201A0AEF70077EC2
:100AC400057F241245129061CD740AF090619774E9
:100AD40001F0020B7B201A077E057F311245127844
:100AE400397C707D017B017A61790312270D752EA3
:100AF400FF752F0575303A7B017A70793912509C55
:100B0400E4F54DF558F554C201D202C2992099FD7D
:100B1400D299906197E004F09061CD7406F080570B
:100B24009061CCE0FFB40106A3743CF08049EFB4BB
:100B3400030A05489061CD743CF0803BEFB4021782
:100B4400E4F548D20CD209F54AC20E906000740B49
:100B5400F0A374B8F08020201A0AEF70077E057F96
:100B6400241245129061CD740AF09061977401F0DB
:100B74008005E4906197F0E49061CCF030020302C8
:100B84000EA0E5086003020EA0200C03020EA0E5EF
:100B940052C394144003020EA0E5496547605A7598
:100BA400F00DE547A424FAF582E5F0346BF583E013
:100BB4002405F528C3940E502E75F00DE547A424A2
:100BC400F6F582E5F0346BF58363A20174042552D3
:100BD400F582E43460F58363A201AF2812388BE513
:100BE400282552F552800A201A077E057F3C1245BB
:100BF40012054753473F020EA075F075E555A4242E
:100C04004EF582E5F03468F583E07003020D0CE5DF
:100C140046705775F075E555A42452F582E5F03415
:100C240068F583E02405F528C3940E502E75F075FD
:100C3400E555A4244EF582E5F03468F58363A201FA
:100C440074042552F582E43460F58363A201AF286D
:100C540012388BE5282552F552800A201A077E05A2
:100C64007F3C1245120546020EA075F075E555A4A9
:100C74002451F582E5F03468F583E0540FFFE5462E
:100C8400D39F506775F075E555A42452F582E5F0BD
:100C94003468F58375F00DE546122639E02405F530
:100CA40028C3940E503675F075E555A4244EF5828C
:100CB400E5F03468F58375F00DE54612263963A234
:100CC4000174042552F582E43460F58363A201AF14
:100CD4002812388BE5282552F552800A201A077EFF
:100CE400057F3C1245120546020EA0E4F54675F058
:100CF40075E555A4244EF582E5F03468F583E4F0F7
:100D04000555535507020EA00555535507E545658E
:100D14005D605A75F00DE55DA424D2F582E5F034EA
:100D240061F583E02405F528C3940E502E75F00D6B
:100D3400E55DA424CEF582E5F03461F58363A20178
:100D440074042552F582E43460F58363A201AF286C
:100D540012388BE5282552F552800A201A077E05A1
:100D64007F3C124512055D535D7F020EA0E553756D
:100D7400F00DA4242BF582E43461F583E06069E589
:100D84005375F00DA4242FF582E43461F583E02437
:100D940005F528C3940E502DE55375F00DA4242BAE
:100DA400F582E43461F58363A20174042552F5826B
:100DB400E43460F58363A201AF2812388BE528255B
:100DC40052F552800A201A077E057F3C124512E52F
:100DD4005375F00DA4242BF582E43461F583E4F01B
:100DE4000553535307020EA0055353530775F06878
:100DF400E55CA4243AF582E5F03471F58375F00DD1
:100E0400E54B122639E07003020E8F75F075E55C30
:100E1400A4245FF582E5F03468F58375F00DE54BA5
:100E2400122639E02405F528C3940E503675F07562
:100E3400E55CA4245BF582E5F03468F58375F00D78
:100E4400E54B12263963A20174042552F582E43479
:100E540060F58363A201AF2812388BE5282552F58B
:100E640052800A201A077E057F3C12451275F068ED
:100E7400E55CA4243AF582E5F03471F58375F00D50
:100E8400E54B122639E4F0054B8011054BE54BC3C5
:100E940094084008E4F54B055C535C0730020302F8
:100EA4000F62E5086003020F62200C03020F62E583
:100EB4004A6401706930071520080D906002F0A3A0
:100EC4007419F07F021248E1C207020F62E5526012
:100ED40029200E26E4906002F0A37419F0E5522450
:100EE40002FF1248E10548200805D20EE4F548E463
:100EF400F552906000F0A3F08064D3906001E09418
:100F0400E8906000E094034055E4F0A3F0300E4E06
:100F1400C20E201A497E057F471245128040E54AD9
:100F2400703C200406754A01F55222D3906001E01A
:100F340094E8906000E094034024E4F0A3F0A374E8
:100F4400FEF0A374A0F0A374FFF07F031248E1E461
:100F5400F5520548201A077E057F57124512E558B9
:100F6400700302110BF528E4F558F54EF54FE5280A
:100F7400547FF551E52854802439F582E4346FF523
:100F84008363A2019005E163A201AF51AE50AD4F5E
:100F9400AC4E1238BE8F518E508D4F8C4EE5285476
:100FA400802439F582E4346FAF82F5298F2A5328DF
:100FB4007F74372528F582E4346FF583E0FEA3E0DF
:100FC400655B7003EE655A702DE528D394044026C2
:100FD400201A077E057F62124512E54CB5281120C0
:100FE4001A077E057F7612451274052548F54822B6
:100FF40074032548F548E54F454E6022301A030234
:10100400110B7E057F80124512E4FBAD28AF2AAE9A
:10101400291246CD7D03AF4FAE4E1245F322201A5E
:101024002CE54A640160147E057F8B124512E4FBB3
:10103400AD28AF2AAE291246CD80127E057F9012CC
:101044004512E4FBAD28AF2AAE291246CDE528B4FB
:101054000406E4F548C20E22852A82852983A3E08A
:1010640024E760302499601F24F0600302110175A5
:101074004A01A2079207E4F552301A0302110B7ECB
:10108400057F9A12451222D207201A7B7E057FA77C
:1010940012451222E54A700B201A6C7E057FB412A9
:1010A400451222852A82852983E030E405E4F54847
:1010B400C20ED207E52824FCF571201A1A7E057F9A
:1010C400D4124512E52A2402FFE43529FEE528243A
:1010D400FCFDE4FB1246CDE571C3940F501BE52AD9
:1010E4002402FFE43529F5838F8263A201907B0BF0
:1010F40063A201AF7112388B22E4F57122201A0722
:071104007E057FDC1245129D
:01110B0022C1
:10497D0002194FE493A3F8E493A34003F68001F2E8
:10498D0008DFF48029E493A3F85407240CC8C3333B
:10499D00C4540F4420C8834004F456800146F6DF0A
:1049AD00E4800B01020408102040809053BEE47E89
:1049BD00019360BCA3FF543F30E509541FFEE493FF
:1049CD00A360010ECF54C025E060A840B8E493A3C6
:1049DD00FAE493A3F8E493A3C8C582C8CAC583CAF1
:1049ED00F0A3C8C582C8CAC583CADFE9DEE780BEA9
:0153C40000E8
:1024B300BB010689828A83E0225002E722BBFE0227
:0924C300E32289828A83E493225A
:1024CC00BB010CE58229F582E5833AF583E02250C5
:1024DC0006E92582F8E622BBFE06E92582F8E2220F
:0D24EC00E58229F582E5833AF583E4932229
:1024F900A3F8E0C5F025F0F0E58215827002158396
:06250900E0C838F0E822F2
:10250F0075F008758200EF2FFFEE33FECD33CDCC83
:10251F0033CCC58233C5829BED9AEC99E582984006
:10252F000CF582EE9BFEED9AFDEC99FC0FD5F0D6E3
:10253F00E4CEFBE4CDFAE4CCF9A88222B800C1B90D
:10254F000059BA002DEC8BF084CFCECDFCE5F0CB4B
:10255F00F97818EF2FFFEE33FEED33FDEC33FCEB84
:10256F0033FB10D703994004EB99FB0FD8E5E4F93F
:10257F00FA227818EF2FFFEE33FEED33FDEC33FC2C
:10258F00C933C910D7059BE99A4007EC9BFCE99A20
:10259F00F90FD8E0E4C9FAE4CCFB2275F010EF2F65
:1025AF00FFEE33FEED33FDCC33CCC833C810D70765
:1025BF009BEC9AE899400AED9BFDEC9AFCE899F8A0
:0E25CF000FD5F0DAE4CDFBE4CCFAE4C8F92233
:0E25DD00C3E49FFFE49EFEE49DFDE49CFC220F
:1025EB00EB9FF5F0EA9E42F0E99D42F0E89C45F046
:0125FB0022BD
:0C25FC00ECF0A3EDF0A3EEF0A3EFF02252
:10260800A8828583F0D083D08212261F12261F123B
:10261800261F12261FE473E493A3C583C5F0C58360
:10262800C8C582C8F0A3C583C5F0C583C8C582C81C
:01263800227F
:0C263900A42582F582E5F03583F58322AC
:10282B00E53B242FF8E6053B22782C302602782F47
:10283B00E475F00112278B0224B3201FEB7F2ED2FD
:10284B001F8018EF540F2490D43440D4FF30230B47
:10285B00EF24BFB41A0050032461FFE53C6002155E
:10286B003C053FE53F7002053E30260D782CE475A4
:10287B00F00112278BEF02272A0250F47403D226A1
:10288B008003E4C226F53B8B2C8A2D892EE4F53C84
:10289B00F53EF53FE53C60077F2012286680F57515
:1028AB003DFFC220C21FC221C222C224C225C227A1
:1028BB00122834FF700D3026057F00122877AF3FAA
:1028CB00AE3E22B4255FC2D5C223122834FF24D0DA
:1028DB00B40A00501A75F00A783C30D50508B6FFDB
:1028EB000106C6A426F620D5047002D22280D92474
:1028FB00CFB41A00EF5004C2E5D223022A77D220BC
:10290B0080C6D21F80C0D22180BCD2D580BAD2243F
:10291B0080B47F201228662021077401B53C00404B
:10292B00F112282BFF12286602289FD227D225806E
:10293B009512282BFB12282BFA12282BF94A4B70D5
:10294B000679487A2B7BFF20212EE53C602A7E00FE
:10295B008E827583001224CC60060EEE653D70F0FE
:10296B00C2D5EBC0E0EAC0E0E9C0E0EE122ABED06F
:10297B00E0F9D0E0FAD0E0FB1224B3FF60AAEBC081
:10298B00E0EAC0E0E9C0E0122866D0E02401F9D00B
:10299B00E03400FAD0E0FBE53D0460DCD53DD980A6
:1029AB00877BFF7A2A79BAD221809C7910800279B1
:1029BB0008C225C2278008D2D5790A8004790AC2B9
:1029CB00D5E53D047002F53DE4FAFDFEFF12282B20
:1029DB00FC7B0820201312282BFD7B10301F0A12C2
:1029EB00282BFE12282BFF7B20EC3382D592D5505F
:1029FB0013C3E4301F069FFFE49EFEE42020039DDB
:102A0B00FDE49CFCE4CBF8C220EC700CCFCECDCC1B
:102A1B00E824F8F870F38017C3EF33FFEE33FEEDC5
:102A2B0033FDEC33FCEB33FB994002FB0FD8E9EBA6
:102A3B00302005F8D0E0C448B220C0E00AEC4D4E7F
:102A4B004F78207B0070C2EAB53D0040BCC0E0125D
:102A5B002AC0D0F0D0E0202004C4C0E0C4B220C013
:102A6B00F012284FD0F0D5F0EB02289F1227EA295D
:102A7B003C5329B658290D4C29094229BA4F29C272
:0F2A8B004429C24929224329C85529AC4629AC00
:102A9A004529AC472B685029112D29152E29382B89
:102AAA002919232936202B512A28D14800002930F8
:102ABA003F3F3F00790AA2D5202214302409B910D9
:102ACA00020404B9080104A2D520250250010420F9
:102ADA0021689221B53C005034C0E07F2030221991
:102AEA007F30A22172257224500F122B17C221C2E5
:102AFA0025C224C2277F30800F302403E9C0E012A8
:102B0A002866302403D0E0F9D0E0B53CCC30241755
:102B1A007F30B9100C1228667F583023077F7880DF
:102B2A0003B908031228663021057F2D0228667F23
:102B3A00202027F87F2B2025F322922180CF286E90
:102B4A00756C6C2900D22012282B3020F8C220780C
:102B5A003C30D50108F60228D12D50434958122895
:102B6A002B2403B405004001E4902B6393122857E9
:0D2B7A00743A122857D222753C040229B685
:10509C008B2B8A2C892D8B318A328933AB2B052DA6
:1050AC00E52DAA2C7002052C14F91224B370ED74A2
:1050BC00FF252DF52D74FF352CF52CAB2E0530E589
:1050CC0030AA2F7002052F14F91224B3FFAB2B0555
:1050DC002DE52DAA2C7002052C14F9EF12272A703D
:0850EC00DAAB31AA32A933222C
:103B11008B2C8A2D892EE4F538F537F536F535F5F8
:103B210033F534E5304531452F6012EBC0E0EAC092
:103B3100E0E9C0E0AB2FAA30A93112279BAB2C05DD
:103B41002EE52EAA2D7002052D14F91224B3F53994
:103B5100C394094007E539D3940D40E1E539642068
:103B610060DBE539B42D054334038016E539B42B08
:103B710005433401800C74FF252EF52E74FF352D7D
:103B8100F52DE53260046410703FAB2CAA2DA92EEF
:103B91001224B364306009E532702E75320A80292F
:103BA1009000011224CCFF64786004EFB4581343F1
:103BB10034017532107402252EF52EE4352DF52DC4
:103BC1008007E5327003753208AB2C052EE52EAA6D
:103BD1002D7002052D14F91224B3F539C3946140F7
:103BE1000AE539D3947A50035339DF74D02539F576
:103BF10039C3940A400CE5399411406D74F92539A3
:103C0100F539E539D39532506043340185383D8526
:103C1100373C85363B85353AAF327E00E4FCFDAB5F
:103C210038AA37A936A83512273CC8ECC8C9EDC94E
:103C3100CAEECACBEFCBE4FCFDFEEB2539F538EE3D
:103C41003AF537ED39F536EC38F535AF38AE37ADF5
:103C510036FCAB3DAA3CA93BA83AD31225EB500355
:103C6100023BCA433404023BCAE53420E003E4804A
:103C71002DE5304531452F601EAB2CE52E24FFF993
:103C8100E52D34FFFAEBC0E0EAC0E0E9C0E0AB2F7C
:103C9100AA30A93112279BE53430E20774FFFFFEF9
:103CA100FDFC22E534AF38AE37AD36AC3530E1033B
:043CB1000225DD22E9
:10264500E709F60870FA8046E709F20870FA803E55
:1026550088828C83E709F0A370FA807CE309F60889
:1026650070FA8074E309F20870FA806C88828C83B2
:10267500E309F0A370FA806089828A83E0A3F608F3
:1026850070FA805489828A83E0A3F20870FA804840
:1026950080D280FA80C680D4806180F2802F80103D
:1026A50080A680EA809A80A880DA80E280CA802F9E
:1026B50089828A8363A20188828C8363A201E49361
:1026C500A363A201F0A363A20170F3800B89828A40
:1026D50083E493A3F60870F9ECFAA9F0EDFB2289DF
:1026E500828A8363A20188828C8363A201E0A3634B
:1026F500A201F0A363A20170F480DD89828A83E4DC
:1027050093A3F20870F980D088F0ED2402B4040098
:1027150050C6F582EB2402B4040050BC2323458245
:052725002390269573CE
:10272A00BB010689828A83F0225002F722BBFE018E
:02273A00F32288
:10273C00E88FF0A4CC8BF0A42CFCE98EF0A42CFC3C
:10274C008AF0EDA42CFCEA8EF0A4CDA8F08BF0A4BA
:10275C002DCC3825F0FDE98FF0A42CCD35F0FCEB19
:10276C008EF0A4FEA9F0EB8FF0A4CFC5F02ECD39DE
:0F277C00FEE43CFCEAA42DCE35F0FDE43CFC224B
:10278B00FAE6FB0808E6F925F0F618E6CA3AF6224F
:10279B00BB011A89828A83D0F0D0E0F8D0E0F9D05F
:1027AB00E0FAD0E0FBE8C0E0C0F00228195016E9CF
:1027BB00F8D083D082D0E0F9D0E0FAD0E0FBC08231
:1027CB00C083022810BBFE16E9F8D083D082D0E07C
:0F27DB00F9D0E0FAD0E0FBC082C08302282222AE
:1027EA00D083D082F8E4937012740193700DA3A37E
:1027FA0093F8740193F5828883E473740293686092
:06280A00EFA3A3A380DF91
:09281000EBF608EAF608E9F622ED
:09281900EBF0A3EAF0A3E9F022C0
:09282200EBF208EAF208E9F222E7
:00000001FF
